:100000009128A2003B200C080D0403198C2886209F
:1000100084132208800664000D280E288C0A031918
:100020008D0F0B2880068C288F002408840022095D
:100030003C2084138F0803198C28F03091000E089F
:1000400080389000F03091030319910003198F0359
:1000500003198C282B283F2003010C1822088E1F1F
:1000600022088E0803190301900F382880061F28E4
:10007000392800002228FF3A841780058C280D08B3
:100080000C0403198C0A80300C1A8D060C198D068D
:100090008C188D060D0D8C0D8D0D8C288F018E000A
:1000A000FF308E07031C8F07031C8C2803308D0044
:1000B000DF305C2050288D01E83E8C008D09FC303B
:1000C000031C65288C07031862288C0764008D0FB9
:1000D00062280C186B288C1C6F2800006F28080001
:1000E000103094008D018C01930C920C031C7E281F
:1000F0000E088C070F0803180F0F8D078D0C8C0C42
:10010000910C900C940B742810088C288C098D0984
:100110008C0A03198D0A08008313031383126400E9
:1001200008008316FF3085000C30860083121E30D5
:10013000AF000530AD000530B2000130B3006400FF
:100140000B3033020318C8280630A4001030A20078
:1001500033089200930103308E008F0170209E00BF
:1001600011089F005A309E0703189F0A1E088E0030
:100170000230142002308606831686100130831266
:10018000860683160610643083124E20B30F9F2814
:10019000942129188614291C86102A1806142A1C52
:1001A000061029089200930102308E008F01702002
:1001B0009E0011089F002A081E07A8002808033C7B
:1001C000031CEA2800308A0028088207832927298F
:1001D0005529EA280630A4001030A2005A308E00BB
:1001E0000130142050308E00023014207D308E00FB
:1001F000013014205A308E000230142064308E00FA
:10020000023014200130B3006400033033020318BD
:100210001B29AA30AE00B8217830AC007830B1008C
:10022000B8216430AE00B821A030AC00A030B100DD
:10023000B821B30F042926088C0027088D003F2021
:100240000C08A6000D08A7006400261855290630E2
:10025000A4001030A2008C308E00013014205030E9
:100260008E00023014207D308E00013014205F306B
:100270008E00023014200130B300640003303302DA
:1002800003185429AA30AE00B8217830AC00A03051
:10029000B100B8216430AE00B821A030AC00783095
:1002A000B100B821B30F3D29C8280630A400103092
:1002B000A2008C308E000130142078308E00023085
:1002C00014206E308E000130142064308E00023015
:1002D00014200130B3006400033033020318822974
:1002E000AA30AE00B821A030AC007830B100B821FF
:1002F0006430AE00B8217830AC00A030B100B82135
:10030000B30F6B29C828AA30AE00B821A030AC00CA
:10031000A030B100B8216430AE00B8217830AC0014
:100320007830B100B821C828AB01B001A901AA01F9
:100330000130B300640033082F02031CA9296400B4
:100340000619A329AB0A64008619A729B00AB30FBE
:100350009A2964002D082B02031CB0290130A90042
:10036000640032083002031CB7290130AA000800DB
:100370000130B40064000B3034020318D8292E0871
:100380008C008D0106308400803001202C088C0008
:100390008D01063084004030012031088C008D0131
:1003A00006308400203001200D304E20B40FBA29D1
:0603B00008006300D929DA
:02400E00F53F7C
:00000001FF
